:020000040000FA
:100000008A150A125B290000F20003088301A00090
:100010000A08A1000408A2000B1900000B18000038
:100020008B180000831203138A110A128C196020A6
:100030000C1B00008C1A00000C1A00000C190000A8
:100040008C1800000C1800000D1800008301220815
:10005000840021088A0020088300F20E720E090035
:1000C000831603171008110583128A110A120319E7
:1000D0008528AB008A110A122B19CF208A110A1227
:1000E0002B1889208A110A12AB19DB208A110A12F7
:1000F000AB1ABB208A110A12AB18C2208A110A124D
:100100002B1AAF208A110A126028831203138C1154
:100110000800AC01C4018316901190119011901148
:100120000830A100B830A2008830A000C030A6007E
:100130000830A40096019001831203138C118316DA
:100140000317063098003B309100FF3093000130D8
:10015000970083120130AD000313031708008316C4
:1001600011121012101111159514831203138C1112
:1001700003174414080083169012831203138C1182
:1001800003170800831690101208130592018312BA
:1001900003138C110317B000831203170800831692
:1001A00011111011101211169510831203138C11D6
:1001B0000317C40108008317831603171408A03E11
:1001C000840083120008A000840A0008A100840AA9
:1001D0000008A2008316031714089011831203135A
:1001E0008C110317C50020083C39B100243A8A114C
:1001F0000A12031928293108043A8A110A1203192C
:1002000008293108343A8A110A1203198A29080088
:1002100045088A110A12031D1D292E08213A8A1148
:100220000A12031D132983160830A1008830A0008C
:100230008A110A12831282290800083A8A110A12C6
:10024000031D232908004508103A03190800080077
:10025000450818398A110A12031D7B292E08063A0F
:100260008A110A12031D38298A110A127E247A295A
:100270002E08663A8A110A12031D44298A110A12AD
:100280007E248A110A127A292E08053A8A110A1246
:10029000031D50298A110A127B238A110A127A2916
:1002A0002E08033A8A110A12031D59298A110A12CB
:1002B0007A292E08013A8A110A12031D7729270884
:1002C000013A8A110A12031D6B298316191483122D
:1002D0008A110A127A292708023A8A110A12031D82
:1002E0007A2983161A1483128A110A127A298A111A
:1002F0000A126A2D0800083A8A110A12031D812980
:100300000800080083160317A501C830A400831253
:10031000AE0108008317220884000008A300840AA5
:100320000008A400840A0008A500840A0008A600AA
:10033000840A0008A700840A0008A800840A0008AC
:10034000A900840A0008AA0083160830A100A400AE
:1003500083122308213A88300319C8308316A0007D
:1003600015128312AE0123088A110A120319E82913
:100370002308013A8A110A120319032A2308023AB0
:100380008A110A120319182A2308803A8A110A12BC
:100390000319242A2308813A8A110A120319362ADA
:1003A0002308823A8A110A120319482A230860395D
:1003B000203A8A110A120319AD2C23086039403AF9
:1003C0008A110A12031D0C2B8A110A12AC2C080088
:1003D0002408013A8A110A120319872B2408053AC6
:1003E0008A110A1203196F2B2408093A8A110A127A
:1003F00003191C2C2408033A8A110A120319CB2B67
:100400008A110A120C2B2408013A8A110A120319C4
:10041000C82B24080B3A8A110A1203196B2C2408E2
:10042000033A8A110A1203190C2C8A110A120C2B96
:100430002408013A8A110A120319922B2408033A5C
:100440008A110A120319D62B2408083A8A110A12B3
:1004500003190F2C2408063A8A110A120319522A8A
:100460002408003A8A110A120319112B24080A3AA7
:100470008A110A1203194D2C2408003A8A110A1213
:100480000319202B2408063A8A110A120319522A4A
:100490002408003A8A110A1203194B2B8A110A12F6
:1004A0000C2B08002608223A8A110A120319012D82
:1004B0002608213A8A110A1203194F2D02308A00A8
:1004C000031026080339673E03188A0A82000C2BA2
:1004D0006B2A852AB52A0630AE000830B500933065
:1004E000B2000530B3008A110A128D25B400AA08A3
:1004F0008A110A12031D802A29022908031CB4004C
:10050000B40A8A110A127E2408000630AE000310D5
:10051000250D8A110A127925B2000310250D013E1E
:100520007925B3000230B2070318B30A8A110A1200
:100530008D25B4000230B202031CB303AA088A114D
:100540000A120319A62A8A110A12AE2A34082902AD
:100550008A110A120318AE2A2908B4000830B5001F
:10056000B40A8A110A127E2408006630AE002708F9
:100570008A110A12031DC62A2808031DC62A4D30F7
:10058000B2000630B3008A110A12FD2A0630B30009
:100590004F30B200BB018A110A121126B20A27029B
:1005A0008A110A12031DDC2A8A110A121126280256
:1005B0008A110A120319E82AB20ABB0A533032021E
:1005C0008A110A12031CCB2AAE018A110A120C2BC3
:1005D000063025028A110A12031CF22AAE018A1182
:1005E0000A120C2B250DB3003B088A110A1217269C
:1005F000B200B30A3B081726B3008A110A1211266B
:10060000B40029022908031CB4000830B500B40A5C
:100610008A110A127E240800831603171814831205
:100620000800831626088400831283172D08800093
:10063000840A800183160230A500C830A400080097
:1006400083161708023A8A110A12031D2D2B8312F2
:1006500027088A110A12031D2D2B83161708033A47
:100660008A110A12031D0C2B83122708003C8A11E1
:100670000A12031C0C2B2708383E8400831700083D
:10068000F000831626088400700880000230A50060
:10069000C830A40008000F302705013A8A110A1259
:1006A0000319602B0F302705023A8A110A12031D25
:1006B0000C2B031083161A1803148A110A12642BC8
:1006C0000310831619180314260884008001800D76
:1006D000840A80010230A500C830A4000800250863
:1006E000AF008A110A12AF1B0C2B8A110A12822149
:1006F0000530AE000800AE01AC012F08831696004D
:100700008A110A120319862B023097000800250867
:10071000013A8A110A12031D0C2BAD108A110A121C
:100720008221080025088A110A12031D0C2B2608B5
:10073000031D0C2B831603301705023A8A110A1287
:10074000031DAD2B83120F302705031DAD2B831620
:1007500018108A110A128221080083160330170527
:10076000033A8A110A12031D0C2B83120F3027053E
:10077000023C8A110A12031C0C2B83170F30270529
:100780008316983E840000108A110A128221080004
:100790008A110A120C2B2508013A8A110A12031D2C
:1007A0000C2BAD148A110A128221080025088A1127
:1007B0000A12031D0C2B2608031D0C2B8316033075
:1007C0001705023A8A110A12031DF12B83120F300A
:1007D0002705031DF12B831618148A110A12822192
:1007E0000800831603301705033A8A110A12031D05
:1007F0000C2B83120F302705023C8A110A12031CAE
:100800000C2B83170F3027058316983E84000014A5
:100810008A110A12822108008A110A120C2B8316EF
:1008200026088400831283172C0880008316013069
:10083000A500C830A40008002508013C8A110A124E
:10084000031C0C2B2508AC008A110A1203192B2C4F
:100850008316033097008A110A1282218316031728
:10086000C830AA000830A9008830A8000830AD00C0
:10087000D030AE004830AC00D830B2000830B10003
:100880008830B0000830B500D830B6004830B40029
:100890000E3099000E309A00080083161708033AAC
:1008A0008A110A12031D0C2B83122708003C8A119F
:1008B0000A12031C0C2B2708383E840083170008FB
:1008C000F000831626088400700880000130A5001F
:1008D000C830A40008008316170883120339033AAE
:1008E0008A110A12031D0C2B2708383E8400831737
:1008F000250880008A110A12822108008316031736
:1009000083172608840083120317B70137083502BE
:100910008A110A120319A02C8A110A12B40B932C03
:100920008A110A129F2C8A110A128D258000B70A9B
:10093000840A8A110A12B20F862CB30A862CAE01E1
:1009400037088316A5004030240640398838A400B3
:0A0950008A110A12080008000800CE
:06095A008A110A122308B5
:10096000213A0319D42C8A110A122308223A0319B6
:10097000712D8A110A122308233A0319712D8A1145
:100980000A122308A13A0319712D8A110A122308A9
:10099000A23A0319712D8A110A122308A33A0319E6
:1009A000712D8A110A120C2B2408013A8A110A129D
:1009B0000319712D2408023A8A110A120319712DA4
:1009C0002408033A8A110A120319712D2408063AE1
:1009D0008A110A120319012D2408093A8A110A12F0
:1009E0000319742D24080A3A8A110A120319712D69
:1009F00024080B3A8A110A120319712D8A110A125E
:100A00000C2B831203170630AE000830B500260801
:100A1000013A8A110A120319202D0310270D8A1199
:100A20000A128325B2000310270D013E8325B3006F
:100A30008A110A128D25B400B20A8A110A12402DB9
:100A40002608023A8A110A120319392D0310270DBC
:100A50008A110A128325B2000310270D013E832557
:100A6000B3008A110A128D25B400B20A8A110A1243
:100A7000402D2608033A8A110A1203190C2B08008C
:100A80002A088A110A12031D4A2D2908340229084E
:100A90000318B400B40A8A110A127E240800063032
:100AA000AE000830B500B730B2000530B3008A118F
:100AB0000A128D25B400AA088A110A12031D642D9A
:100AC00029022908031CB400B40A8A110A127E24E0
:100AD000080008008A110A122E08063A03197E241B
:100AE00008008A110A120C2B2130AE00831603175E
:100AF0000800F00005308A008130700703188A0A68
:100B00008200A5340534F00005308A008B30700770
:100B100003188A0A8200C734053483120317330886
:100B20008A00320882001234013400340134003467
:100B30000034003408340034003404340034003409
:100B400000340234013400340134093402342234D4
:100B50000034013401340434803432340934043430
:100B600000340034013403340034003400340934D8
:100B70002134003401340034013422344934003447
:100B80000734053481340334083400340A344934DA
:100B9000053401341534003409340434A1340134EB
:100BA00009340134A1340034093430340934313487
:100BB0001534813425347F34753408349534023447
:100BC00081340234053402340934BA340934BB3474
:100BD00081340234C03416340134FE340534013417
:100BE000093432341534813425347F347534083473
:100BF0009534013481340234053409341934013414
:100C00002934183415340034253401347534013452
:100C1000953418345534003465340034813402344A
:100C2000C0348312031733088A0032088200F000B0
:100C30000310F00D8A110A122A26B600F00A8A1152
:100C40000A122A26F00070088A00360833070318B3
:100C50008A0A820006308A003130700703188A0A37
:100C6000820035340634413406344D34063453346E
:100C7000063475340634913406349D340634A73472
:100C800006344D340634B7340634CB340634F934E4
:100C90000634053407340F3407340634033409347A
:100CA00004340434083422340334493400344F34D7
:100CB000003443340034613400347234003464341A
:100CC00000342D340034553400345334003442346D
:100CD00000344134003478340034653400347334E3
:100CE000003420340034203400341C3403344D34B8
:100CF0000034613400346E340034753400346534AB
:100D000000346C34003420340034563400346534FC
:100D100000346C340034653400347A3400342034C8
:100D200000340C34033456340034313400342E345F
:100D3000003430340034303400340A340334433463
:100D400000346634003467340034313400341034F5
:100D500003344E3400346F34003474340034683457
:100D60000034693400346E34003467340034143491
:100D700003344D3400346934003463340034723445
:100D800000346F3400346334003468340034693420
:100D90000034703400342E34033450340034693459
:100DA0000034633400343134003436340034433496
:100DB00000343734003436340034353400342034D1
:100DC0000034553400345334003442340034203479
:100DD0000034493400344F34003443340034613437
:100DE00000347234003464340034733400342034FA
:100DF00000340C34033456340034313400342E348F
:100E0000003430340034303400340A340334433492
:100E10000034663400346734003431340034103424
:100E200003344E3400346F34003474340034683486
:0E0E30000034693400346E340034673400340A
:10100000030883120317C3000408BD0083160317E7
:101010008A150A12A81B3C28290883120317C1004D
:10102000C2008A150A1203192C28831603172A08EE
:1010300083120317BE0083173E0884000008F100E6
:101040003D088400C31F831371088000BD0ABE0AD7
:101050008A150A12C10B1B28831628084039403A0A
:101060008838A8000830A90083124208F10043081C
:1010700083007108031408008312031743088300D8
:1010800003100800030883120317C3000408BD00FF
:10109000831603178A150A12B01B7E2831088312A3
:1010A0000317C100C2008A150A1203196E2883169D
:1010B0000317320883120317BE0083173E0884000B
:1010C0000008F1003D088400C31F831371088000ED
:1010D000BD0ABE0A8A150A12C10B5D2883163008A4
:1010E0004039403A8838B0000830B10083124208D5
:1010F000F1004308830071080314080083120317EA
:101100004308830003100800F1000308831203174B
:10111000C30071080F39C1000408BE0041088316DE
:1011200003178A150A12AC1BBB28AD008A150A12D8
:101130000319AF282E088312BD008317C31F831322
:101140003E0884000008F10083173D088400710800
:101150008000BD0ABE0A8A150A12C10B9D2883169B
:101160002C084039403A8838AC00831203174308F2
:1011700083000314080003100800F1000308831221
:101180000317C30071080F39C1000408BE004108ED
:10119000831603178A150A12B41BF428B5008A15A2
:1011A0000A120319E82836088312BD008317C31FEB
:1011B00083133E0884000008F10083173D08840073
:1011C00071088000BD0ABE0A8A150A12C10BD62812
:1011D000831634084039403A8838B4008312031724
:1011E0004308830003140800031008008317033921
:1011F000983E84000014080083170339983E840049
:101200000010080083120317441C080083161011F5
:10121000111595146300000095101012111610118D
:101220001111080083120317AD1C080083169510D6
:10123000111610121111101115158312BB018030F7
:10124000BC008A150A12BB0B2329BC0B2329831669
:10125000151108008316031795118312BC01BB01F9
:101260008A150A12BB0F3229BC0F32298A150A12BD
:101270003A2108008316031797010130910090016D
:10128000083095008312AC010130AD00B801B901FE
:10129000BA01FF30AE00831203138C1183168C1534
:1012A0000B178B17080083160317951195149701D8
:0612B00003138C1108007D
:0A12B6001E30F200F20B5D298316D2
:1012C000031381178A150A123A21831603178A1508
:1012D0000A12640003301705033A031D69298312BB
:1012E00003138501860187018A150A123D228312A4
:1012F00003130516FF30F400FF30F5008A150A12BB
:10130000831323308400083000208A150A12F50B5D
:101310007E298A150A12F40B7C2983120313051205
:101320008A150A12831323308400083000208312A8
:10133000031381018312031381309F0080221F1544
:101340008A150A121F19A0291E08A300FF3A0319C3
:10135000A3037F30A302802283120313810183122F
:10136000031389309F0080221F158A150A121F1946
:10137000B5291E08A400FF3A0319A4037F30A40274
:1013800080228312031381018312031391309F0083
:1013900080221F158A150A121F19CA291E08A500C6
:1013A000FF3A0319A5037F30A5028022831203139D
:1013B00081018312031399309F0080221F158A1523
:1013C0000A121F19DF291E08A600FF3A0319A603F7
:1013D0007F30A6028022831203138101831203133C
:1013E000A1309F0080221F158A150A121F19F429A7
:1013F0001E08A700FF3A0319A7037F30A702802227
:10140000831603130630870083120313003087000E
:101410000000000000000608A800A80983160313B6
:10142000053087008312031300308700000000009E
:1014300000000608A900A9098316031303308700DA
:10144000831203130030870000000000000006082C
:10145000AA00AA098A150A128313831203132330E0
:101460008400083084208A150A12031C2A2A8A154F
:101470000A1271228A150A12902983160313EF307B
:101480008500FF3086000730870083160313811321
:101490008316031302309F00831203139F171F1339
:1014A000831603130C1383120313A301A401A501D4
:1014B000A601A701A801A901AA010800FF30831213
:1014C0000313F40000008A150A12F40B622A0800C4
:1014D00083120313FF30F4008A150A12F40B6C2AEE
:1014E00008001430F400FF30F500000000008A15F9
:1014F0000A12F50B752A8A150A12F40B732A0800D2
:101500000230F400FF30F500000000008A150A12D6
:0E151000F50B842A8A150A12F40B822A0800B1
:044000000034003454
:02400E00FA3F77
:00000001FF
